:020000040000FA
:020000000528D1
:08000800090083160313003008
:100010008600133085009B0107309C008B01831202
:10002000031386014430DF00D4011C30E000600877
:100030004D21DF002030540784005F08FF39031989
:1000400025288000D40AE00A17280B21E001600867
:1000500044210B210C30E00044210A30DE00013045
:10006000E0000310E620AE2060088600AE20860186
:10007000A72060088600AE208601E00D031C322810
:10008000DE03031D2F28E620003056302030DA0032
:100090000430D900D401E620A720A720D5018A0189
:1000A0005A0854073F39203884000008E03ED30046
:1000B000D201CD3E03185214D21452088A005308BC
:1000C0000310D30DD30DD3075218D30A5308D80009
:1000D00055085807521C0022521800238600A02001
:1000E0008601D50A5508053C031D6828A020A020DC
:1000F000A020D40A541E4E28D90B4A28DA0A5A08DE
:100100003F392038DA002E30F92048282030DB0033
:10011000DB0B882808001030DB00DB0B8D28080083
:10012000912892280130DB000130DC000430DD0032
:10013000DF280130DB000130DC001330DD00DF2878
:100140000130DB000130DC002630DD00DF2801302B
:10015000DB000130DC00C830DD00DF280130DB00CF
:100160000430DC00E630DD00DF280130DB00083041
:10017000DC00CD30DD00DF280130DB001430DC0096
:100180008030DD00DF280130DB004F30DC00013043
:10019000DD00DF280130DB00C430DC000230DD0090
:1001A000DF280430DB000E30DC003830DD00DF28D3
:1001B0000830DB00A130DC00DA30DD00DF28DD0BA9
:1001C000DF28DC0BDF28DB0BDF2808000518E6281A
:1001D000051CE828AE200800DF010830DE0086207C
:1001E0000310051A0314DF0CDE0BEF28862086208F
:1001F0000800E1000830DE0085118620E10C0318BC
:1002000003298511042985158620DE0BFE28851516
:100210008620862008000D3010210A3010210800A9
:10022000F92008006008E6208D00831603130C14E3
:10023000831203130C0883120313DF00FF39031D1D
:10024000222908000530D50020305F02D300D201FA
:10025000CD3E03185214D21452088A00D30DD30D88
:10026000D3075508053C5307521C0022521800239F
:100270008600A0208A01D50B242900308600A0200A
:10028000A020E00A1229080060084D21E00AFF3989
:1002900003190800102144290800831203178D0058
:1002A000831603178C130C14831203170C08831284
:1002B000031308008D00831603130C148312031319
:1002C0000C08831203130800031783128C008B138E
:1002D00083168C130C1555308D00AA308D008C14AC
:1002E0008B170C118C1872290C128312031308003F
:1002F00000000000000000000000000000000000FE
:1003000000000000000000000000000000000000ED
:1003100000000000000000000000000000000000DD
:1003200000000000000000000000000000000000CD
:1003300000000000000000000000000000000000BD
:1003400000000000000000000000000000000000AD
:10035000000000000000000000000000000000009D
:10036000000000000000000000000000000000008D
:10037000000000000000000000000000000000007D
:10038000000000000000000000000000000000006D
:10039000000000000000000000000000000000005D
:1003A000000000000000000000000000000000004D
:1003B000000000000000000000000000000000003D
:1003C000000000000000000000000000000000002D
:1003D000000000000000000000000000000000001D
:1003E000000000000000000000000000000000000D
:0E03F0000000000000000000000000000000FF
:1004000082070034003400340034003400340034F7
:100410004F340034003400340734003407340034DF
:1004200014347F3414347F34143424342A347F3425
:100430002A341234233413340834643462343634A6
:1004400049345534223450340034053403340034F4
:1004500000341C342234413400340034003400347D
:10046000413422341C34143408343E3408341434F7
:10047000083408343E3408340834003450343034FE
:1004800000340034083408340834083408340034A4
:1004900060346034003400342034103408340434C0
:1004A00002343E345134493445343E34003442340D
:1004B0007F3440340034423461345134493446345A
:1004C0002134413445344B3431341834143412342B
:1004D0007F341034273445344534453439343C3482
:1004E0004A344934493430340134713409340534E0
:1004F00003343634493449344934363406344934C3
:10050000493429341E34003436343634003400344F
:100510000034563436340034003408341434223471
:100520004134003414341434143414341434003486
:10053000413422341434083402340134513409343F
:10054000063432344934793441343E347E34113403
:10055000113411347E347F344934493449343634CB
:100560003E3441344134413422347F3441344134C7
:1005700022341C347F3449344934493441347F3483
:1005800009340934093401343E344134493449349E
:100590007A347F340834083408347F3400344134EA
:1005A0007F34413400342034403441343F3401340A
:1005B0007F3408341434223441347F34403440349E
:1005C000403440347F3402340C3402347F347F347E
:1005D0000434083410347F343E34413441344134DF
:1005E0003E347F3409340934093406343E3441340E
:1005F000513421345E347F3409341934293446347B
:1006000082074634493449344934313401340134A1
:100610007F34013401343F344034403440343F347B
:100620001F342034403420341F343F3440343834B5
:1006300040343F346334143408341434633407349E
:100640000834703408340734613451344934453443
:1006500043347F34413441340034003402340434B0
:1006600008341034203400340034413441347F34B1
:10067000043402340134023404344034403440340D
:100680004034403400340134023404340034203423
:1006900054345434543478347F34483444344434F7
:1006A00038343834443444344434203438344434D2
:1006B000443448347F343834543454345434183443
:1006C00008347E340934013402340C345234523448
:1006D00052343E347F3408340434043478340034E3
:1006E00044347D34403400340034203440344434C5
:1006F0003D347F34103428344434003400344134E1
:100700007F34403400347C34043418340434783476
:100710007C34083404340434783438344434443475
:10072000443438347C3414341434143408340834E5
:100730001434143418347C347C34083404340434D1
:1007400008344834543454345434203404343F345A
:100750004434403420343C344034403420347C34FD
:100760001C342034403420341C343C344034303485
:1007700040343C34443428341034283444340C3469
:100780005034503450343C344434643454344C3455
:1007900044340834363441340034003400340034F6
:1007A0007F340034003400340034413436340834AB
:0A07B0000034083404340834043423
:02400E00023F6F
:02401000FC3F73
:1042000048344134503452343834383461342E34E4
:10421000613473346D3420343134363446343834B8
:1042200038345F34783478345F3430343634313471
:104230003034313431340034203450346134753406
:104240006C3446346A3475346A346F342034413403
:104250005234533454345A342034313432343334B5
:104260003434353436343734383439343034313406
:104270003234333434343534363400342034413439
:104280004234433444344534463447344834493462
:104290004A344B344C344D344E344F342034503443
:1042A00051345234533454345534563457345834CA
:1042B00059345A34203461346234633420346434E1
:1042C000653466346734683469346A346B346C340A
:1042D0006D346E346F34703471347234203473340E
:1042E0007434753476347734783479347A342034CD
:0842F00045344E34443400341F
:00000001FF
